:101A400017C01A3A4005930B0902120001010080E9
:101A50003209040000000000000012011001FF0024
:101A60000008D01653070302000000010403090414
:101A7000112420E0A0E6B0E001C01D92AC38B2070E
:101A8000E1F776C1A82FB92F80E090E041E050EA5D
:101A9000609530E009C02D9182279795879510F0C9
:101AA00084279527305EC8F36F5FA8F30895EADFB7
:101AB0008D939D930895CF93CFB7CF93DF93C39525
:101AC000B39BE9F7B39B0BC0B39B09C0B39B07C0A3
:101AD000B39B05C0B39B03C0B39B01C08FC06F9382
:101AE000C0916E00DD27CA58DF4F2F9365E5B39B89
:101AF00003C02F916F91E6CF0F931F934F9320E078
:101B000040E15F9306B3087103FB27F93F9350E070
:101B10003BE039C0187140642F77012F5F5F1EC012
:101B2000406816B318712F7752501FC0406406B337
:101B30002F770871D1F15F5F00C023C0406216B3F8
:101B40002F77187191F15F5F00C025C008711027D1
:101B5000515012F45D5F0000115027952C3F16B3D1
:101B6000C8F618710127015027952C3FC8F6422767
:101B7000499306B3087110274F73115027952C3FD6
:101B8000A8F64695469516B3187179F001270150CD
:101B900027952C3F98F66B5A60F3315006B3B0F698
:101BA00000C010E21ABF00271DC03B503195C31B77
:101BB000D04010E21ABF0881033C29F10B3419F11F
:101BC00020916C001981110F1213EDCF093651F1DC
:101BD0000D3211F0013E39F7CAE01AB715FD02C007
:101BE000CA95D9F7009374003F915F914F911F916F
:101BF0000F912F916F91CAB7C5FD61CFDF91CF9142
:101C0000CFBFCF91089520917400222369F31091E2
:101C10007200112309F534300AF1309372002093D9
:101C20006D001CC0009172000130B4F40AE53091DF
:101C30006F0034FD14C000936F00C1E6D0E013C004
:101C4000052710E000C0000008BB1AC0052710E0FF
:101C5000221F1DC010E021C04AE502C032ED432F13
:101C6000C4E1D0E032E017B31861C39A08B317BBE0
:101C700058E120E865E320FF052708BB2795179565
:101C80001C3FF0F66695B8F7B1F720FF052708BBB3
:101C9000279517951C3FD0F62795179517FF052711
:101CA00000001C3F08BBB0F629913A9519F7077E52
:101CB00010917300110FC651D04008BB11F0109362
:101CC0006C0010E21ABF086017B3177E402F477EE2
:101CD00054E05A95F1F708BB17BB48BB85CF2FEFEF
:101CE000B0E8A0E04AE0B1BF00008DE79CE0B39906
:101CF000FECFB39BFECF0197B399FDCF97FF03C0F3
:101D0000BA1B819501C0BA0FA69539F4A0E428F456
:101D1000281710F031B7282FA1E0415021F731BF2B
:101D200000000895F20121E00C0120935700E8958E
:101D30001124C20102962C01089514BE88E181BDD0
:101D400087E081BDBB9A2FEF85EA9EE0215080405D
:101D50009040E1F700C00000BB988AE580936F00D7
:101D60008FEF80936000AC9A8BB780628BBF089531
:101D7000E4DF712C312C412C512CC5EDD4E114E65B
:101D800086B3887109F014E6115029F4109273009B
:101D900010926C00A4DF0AB605FE05C08CDE80E25E
:101DA0008ABF712C04C0219759F7C0E0D0E0A895F4
:101DB00022E032120CC0E0E4FAE1E054F10983E0E1
:101DC00080935700E8953097C1F7412C512C832D13
:101DD000803459F4F2013297E0348AE1F80750F484
:101DE00085E080935700E89505C0843019F4CD2B29
:101DF00011F4EAC0312C80917200835087FD99C0A4
:101E000090916D009D3209F092C0883009F08FC02A
:101E100083EC809361008AE580936F008091770066
:101E2000807690917800882379F1911108C082E43E
:101E30009AE1909371008093700086E06DC09130BC
:101E400069F441145104F1F080917B00807C482EAC
:101E500050907C0081E187BFE89514C0933081F4F5
:101E60008091790090917A005DDF80917B00909164
:101E70007C0058DF842D8F7329F490E4392E4CC0F8
:101E80009F73392E80E048C08091790010926A00DB
:101E9000911106C010926B002AE630E082E038C053
:101EA000953019F48093730025C09630E9F4909131
:101EB0007A00913019F48AE59AE104C0923041F435
:101EC00088E49AE1909371008093700082E124C0CD
:101ED0009330C1F68111D6CF8CE69AE190937100D0
:101EE0008093700084E018C0983079F0993031F414
:101EF000809375002AE630E080E00AC081E09A30E5
:101F000009F080E02AE630E003C025E730E081E018
:101F1000309371002093700090917E00911105C064
:101F200090917D00981708F4892F8093600010929B
:101F3000720080916F0084FF31C0809160008F3FFC
:101F400069F1C82F893008F0C8E08C1B80936000CD
:101F50009091610088E8892780936100CC2391F0FB
:101F600080917000A2E6B0E0E82FF09171009491AA
:101F70009D9331969C2F980F9E13F9CFF09371008B
:101F8000E09370006C2F82E690E091DDCC5FCC3066
:101F900019F08FEF80936000C0936F00C30101962A
:101FA0003C01803B944029F4EDE3FAE1E491EF3FFA
:101FB00059F40AB605FEE1CE8CE1B39B8CE1815069
:101FC000E1F780E28ABFD9CEB8DE1BBE15BA36CDA6
:021FD000FFCF41
:0400000300001A409F
:00000001FF
